:0400000000001B28B9
:08000800AC00030EAB008312F3
:100010000C180F282B0E8300AC0E2C0E09000C10B0
:10002000AD08031DAD03AE08031DAE032B308E00DB
:10003000CF308F000A280313831600308700831205
:1000400087018316DB308500C830860083128A2240
:100050007C263D2308250C250130612528309C2273
:100060003F24003E031D5124CF24031D3928C524FD
:1000700042280C250330612528309C228230D10093
:10008000D200D3000C2550105C21CF208400033A0D
:1000900003199728501004080F39B300040E0F39C4
:1000A000840093210408AD2103185B285010B3206D
:1000B0000319692890280130B3000121031C652829
:1000C0000230B3000121031887285010B320031D0C
:1000D00083282108A122A1002308A122A30022082D
:1000E000A122A2003308A325B825CB26D6250830A7
:1000F0003306031D44280310470C4707A500A4013D
:10010000CB26DD2544283308A325B8259428BA2317
:10011000031C8C28BA20442850100830B3007228E1
:100120003D233308A325B825CB26CD2544284A23D3
:100130008400033A031D9D285B28501004080F39E2
:10014000B300040E0F398400C4200408A021040861
:100150000C22031887283D233308A325B825CB2676
:100160008225C92044283308063A031908003308B9
:10017000073A08005018080050143D230C2503309E
:10018000A325C420B82508002A30A300A200A1009E
:1001900008000530AD00AD08031DCB280800B201F2
:1001A00032302F02031CDA28E6302F02031CFF280E
:1001B0003214DE2819302F02031CFF28323030029F
:1001C000031CE828E6303002031CFF28B214EC2898
:1001D00019303002031CFF2832303102031CF6288C
:1001E000E6303102031CFF283215FA28193031029B
:1001F000031CFF2807308A003208F8270800033064
:1002000008000030C1004530A1000130BF0042307D
:10021000A2000230C0004330A300AF22031C08003C
:100220000030C1004530A1000130C0004330A200C1
:100230000230BF004230A300AF22031C0800003090
:10024000C0004330A1000130BF004230A2000230A4
:10025000C1004530A300AF22031C08000030C000DD
:100260004330A1000130C1004530A2000230BF0080
:100270004230A300AF22031C08000030BF00423010
:10028000A1000130C0004330A2000230C10045305F
:10029000A300AF22031C08000030BF004230A100C1
:1002A0000130C1004530A2000230C0004330A3003D
:1002B000AF22031C0800080030308126113081264F
:1002C000123081261030AE260130AE260230AE2626
:1002D00000301426AF0001301426AF021030812602
:1002E00031308126123081260030AE261130AE2604
:1002F0000230AE2601301426B00000301426B002C1
:100300001030812611308126323081260030AE2611
:100310000130AE261230AE2602301426B100003075
:100320001426B102080084008408423003199C2975
:10033000041C9E29A2000800A1000800A3000800D8
:100340008400840847300319A929041CAB29A200A2
:100350000800A1000800A30008008400BF00BF0837
:10036000031DCF290030BF004230A1000130C10081
:100370004530A2000230C0004330A300AF22031C6E
:1003800008000030BF004230A1000130C0004330FF
:10039000A2000230C1004530A300AF2208003F1C7C
:1003A000EF290030C0004330A1000130BF004230CF
:1003B000A2000230C1004530A300AF22031C080098
:1003C0000030C1004530A1000130BF004230A20022
:1003D0000230C0004330A300AF22031C08000030ED
:1003E000C1004530A1000130C0004330A2000230FE
:1003F000BF004230A300AF22031C08000030C00041
:100400004330A1000130C1004530A2000230BF00DE
:100410004230A300AF2208008400BF00043033063E
:10042000031D182A1030BE00BC000030BD001D2A7C
:100430000030BE00BC001030BD00840803193A2A09
:10044000041C2E2A5208D500413081263C08013870
:10045000AE260230B4000030B500452A5108D50060
:10046000423081263C080238AE260030B40001300C
:10047000B500452A5308D500403081263C08003895
:10048000AE260230B4000130B500103034048126AD
:100490003E083404AE261030350481263D0835046C
:1004A000AE2634082F26CD000408CC0035082F26B0
:1004B000CF000408CE000430330603196B2A4D0820
:1004C00084004F08CD000408CF004C0884004E087B
:1004D000CC000408CE004F084D02F4004E08031C67
:1004E0004E0F4C02F3007D225508FE240310A40891
:1004F000031D080025080A3C08007D30F700272767
:100500004F08F8004E08F70047277408A400750844
:10051000A5000800901190121012101590102B30A9
:100520008E00CF308F00101483160C1483128B179B
:100530000B172830AE000800AD00AD08031D9D2A42
:100540000800840045300406031953344230040681
:1005500003194734433004060319443408000130BA
:100560003306031DB82A1030BE00BC000030BC2A80
:100570000030BE00BC001030BD00D600103040047A
:1005800081263E084004AE262030410481263D08E5
:100590004104AE2640303F0481263C083F04AE268D
:1005A000542554253F081426C300C3094308C4003A
:1005B000C50041081426C200C2080319392BC20A1B
:1005C0000319392BC20356083F04AE26542554257F
:1005D0003F081426C600C40241081426D700C202F0
:1005E000013033060319002B0318392BD709CD30FE
:1005F00057070318392B5E30F700C309C209082BCF
:10060000031C392BCD3057070318392B6130F70005
:100610004508FC3E0318222B4608FC3E0318222BFB
:100620004208F53E031C392BC209420DA500A40166
:100630000318A40A013033060630031D0730B30047
:1006400003100800F3014208F40027274308F800CC
:10065000F70147277408A4007508A5002408FC3E8C
:10066000031808000030A407031D08002508143CE7
:100670000800A401A501031408000030AE260130D3
:10068000AE260230AE2640308126413081264230EF
:1006900081260800C901CA01CB0100307523031867
:1006A0000334013075230318033402307523031813
:1006B000033402304906031D03344B0303196C2B2A
:1006C0004A03031D03340130320603190434023097
:1006D0003206031914342434013032060319053468
:1006E00002303206031915342534D800D808031D0A
:1006F0007D2B0130D8002F08872B5803031D842B36
:100700000230D8003008872B0430D800310884002C
:10071000A323003803140319080084005809B20504
:100720000408013A031D972BC90A03100800580852
:10073000B2040408023A0319CB0A0408033A031965
:10074000CA0A0310080019300402031CB42BFA3043
:100750000402031802341E300402031C0034323039
:100760000402031C0334003405300402031C00346B
:1007700001340034AE08031DC12B2830AE00023016
:10078000D006D01CCA2B1030812631308126123081
:100790008126D02B303081263130812612308126BF
:1007A0001030AE261130AE260230AE2601301426AF
:1007B000FF3A031D212C00301426AF00023014260E
:1007C000C700AF02D01CEB2B1030812631308126C0
:1007D00012308126F12B10308126313081263230C3
:1007E00081260030AE261130AE261230AE26013002
:1007F0001426FF3A031D212C02301426B1000030CC
:100800001426C800B1022F08C83C0318152C310863
:10081000C83C031C212C4B30A1003C30A2004130CD
:10082000A3004808C7003108232C3108C83C03182E
:10083000212C4130A1003E30A2004B30A3002F08F4
:10084000232C0314080084005208F7004708F40022
:10085000F30127277D30F800F701472775080402C8
:10086000F300F4016430F70027273330F800F70174
:1008700047277308A4007408A5000310080030304F
:10088000812631308126323081260030AE2601307B
:10089000AE260230AE26023014260A3C031C013478
:1008A00000340C25023061253F24003E031D542CEA
:1008B0000C251030812611308126423081261030DF
:1008C000AE260130AE260230AE2600306326C024AC
:1008D00001306326BB24F6242508D100CB268401F1
:1008E00004148C2532309C22103081264130812620
:1008F000123081261030AE260130AE260230AE26F0
:1009000000306326C02402306326BB24F624250869
:10091000D200CB26840184148C2532309C224030B6
:10092000812611308126123081260030AE2611300A
:10093000AE260230AE2601306326C0240230632684
:10094000BB24F6242508D300CB26840104158C256E
:1009500032309C22510884000030D3245208840095
:100960000130D324530884000230D324553084004E
:100970000330D32408002508CF002408CE00080047
:100980002508CD002408CC0008000030E924D1005F
:100990000130E924D2000230E924D30008000330FA
:1009A000E924553A0800831203178D0004088C00CF
:1009B000831603178C130C158B1355308D00AA303A
:1009C0008D008C148B170C118C18E42C83120313DC
:1009D0000800831203178D00831603178C130C1461
:1009E000831203170C088312031308004D08F40048
:1009F0004C08F3007D227D30FE240800A502031878
:100A0000072DA4080319062DA403072DA50108002E
:100A10000430D9003B250800013033255425080057
:100A2000803833250800F10007108710071187115F
:100A3000F11B0714711B8714F11A0715711A87151A
:100A40008516222D85120710871007118711F119BD
:100A5000071471198714F118071571188715851671
:100A6000312D85120800871313255C250800871790
:100A700013255C25080007108710071187118713BD
:100A80008512542533303325333033253230332526
:100A90002C303325063033250C30332501303325F7
:100AA00002303325542508000330F100F201F20B27
:100AB000572DF10B562D08000C30F200F20B5E2D75
:100AC0000800A00000301025840107308A000230A1
:100AD00020060319772D013020060319742D0330E9
:100AE000200603197A2D08000408B5277C2D040878
:100AF000C1277C2D0408C6270038031908003725B4
:100B0000840A672D0A301025723037253D3037258D
:100B1000F925F43037250800013010252D30372510
:100B2000003010254D30041D473037250230102588
:100B3000443004184D30372540301025F925002663
:100B4000F430372508008400840304080310840D62
:100B5000840D840707308A000530A000003010257E
:100B60000408CF273725840AA003031DB02D0800F1
:100B700044301025210837252D3037252208372508
:100B80002D303725230837254A301025002600262A
:100B9000002600260026002608000A301025E23034
:100BA00037253D303725F925002608000A30102565
:100BB000F42500265630372508004B301025D01C70
:100BC000E62D2808372527083725EE2D4A30102531
:100BD000270837252E3037252608372500266D3083
:100BE0003725413037250800280837252E3037258E
:100BF000FB2D280837252708372526083725080024
:100C0000203037250800840019300402031C0E2E02
:100C1000643004020318112E031408000315031096
:100C2000080003110310080084000230DA00831664
:100C300004309F00831284080319242E041C222EE2
:100C40000930252E0130252E19309F00C526C526D6
:100C50001F151F19292EDA0B172E1E0808008400F5
:100C6000831684309F008312840803193D2E041CD0
:100C70003B2E09303E2E01303E2E19308400A50156
:100C8000A4011030AA0004089F00C5261F151F19D3
:100C9000472E83161E088312A5070318A40A1E08F0
:100CA000A407AA0B432E0310A40CA50C0310A40C3C
:100CB000A50C0310A40CA50C0310A40CA50C24086F
:100CC000840025080800A00020081426F03C031C1E
:100CD000642E20082F26F8000408F70020082F268D
:100CE000F4000408F30078087406031D642E7708E6
:100CF0007306031D642E0800831604309F008312C0
:100D00000800840007308A00040E0739041C942E62
:100D10008400AB300407AB278400051106110418CA
:100D20000515841806150800841CA22E8400A63020
:100D30000407A627840006128612041806168418D3
:100D4000861608008400B0300407B027840086109F
:100D5000061004188614841806140800A000201C2D
:100D6000B72E201EB52E0716080007120800A01C7B
:100D7000BF2E201EBD2E0717080007130800201ED7
:100D8000C32E87160800871208005C255C255C25A9
:100D90005C255C250800A601A701A8010130A90077
:100DA000AA00290825050319EF2E07308A0085308F
:100DB0002A078527A60790302A079027A7079B3088
:100DC0002A079B27A8070A302602031CE92EA70A38
:100DD000A6000A302702031CEF2EA80AA7000A303B
:100DE0002A020318FE2EA91FFA2E0130A90024089A
:100DF000A500FC2E0310A90DAA0AD12EA901A8084E
:100E0000031D072F0130A9002030A800092F303022
:100E1000A807A708031D122FA9080319122F2030B5
:100E2000A700142F3030A7073030A6070800F20DB6
:100E3000F10D78080800F20777080318770FF1071B
:100E40000800F2027708031C770FF1020800F50191
:100E50007308FA007408FB000830FC00F70C031854
:100E6000362FFC0B2E2FF301F40100340310412F19
:100E7000F70C031C412F7B08F4077A0803187A0F3C
:100E8000F307F30CF40CF50CFC0B382F0034F101D4
:100E9000F20178082127F30D0730FC00730D1727A6
:100EA000731C542F2127552F1B27F30DFC0B4E2F9E
:100EB000740D1727731C5E2F21275F2F1B27F40D3E
:100EC0000730FC00740D1727741C682F2127692F29
:100ED0001B27F40DFC0B622F750D1727741C722F46
:100EE0002127732F1B27F50D0730FC00750D1727E1
:100EF000751C7C2F21277D2F1B27F50DFC0B762FD2
:100F00007518842F78081B270034820001340234BE
:100F10000434083406340234043408340634023409
:100F200082000034003400340034013403340634C9
:100F300002340534013482000034003400340034BB
:100F400000340034003401340234053482000334A8
:100F5000023401340034820003340234013400349A
:100F600082000334023401340034820754343434B0
:100F70003034303431342034563431342E34333438
:100F800000348207433441344C3400348207453402
:100F9000523452342034433441344C3400348207C8
:100FA0004E3450344E342034203450344E34503487
:100FB000203420343F3420342034203420344E3444
:100FC0004A3446344534543450344A344634453433
:100FD00054344E344D344F345334203450344D3423
:100FE0004F3453342034443449344F34443445343A
:100FF0008207033402341234213422341134013490
:021000000334B7
:00000001FF
